:0E0000000202AD2074726D3130352002006EA8
:0100130032BA
:03001B0002006D73
:200023000200A241545A0D00415445300D0041542B434D45433D320D0041542B434B5044D0
:200043003D0041542B434D45523D332C322C302C302C300D004F4B004552524F520023350E
:20006300002334002A3130352A0032C0E0C0D0758C8B758A7AE52C6002152C152DE52414C2
:200083007004C3B30198147003C30198E52DA2E330B202A2E592B3B39282D0D0D0E032C0A7
:2000A300E0C0D0309818C298E599B4200201C5B40D0201C5B40A0201C51200FA01C5C2993D
:2000C300C202D0D0D0E032752C0201D7752C7801D7752C28E52C70FC22752C7890005812F0
:2000E300028F40026005E52C70F2D3227B3A7C000000DCFCDBF822A92EF7052EA92EB94886
:20010300167931E719F70909B949F8752E47152FA92FB92F02052F22C000C2ACA82FE66088
:2001230002052FD2ACD00022C000C2AC752E30752F30A82E760008B849FAD2ACD00022E49E
:2001430093600612014DA32142222002FDF599D20222C083C08290003C120142D082D0832D
:20016300120142740D12014D12012B1200DC1200CA229001FF12028F40077003743022E485
:200183002290020B12028F400374312290021712028F400374322290022312028F4003748A
:2001A300332290022F12028F400374342290023B12028F400374352290024712028F400339
:2001C30074362290025312028F400374372290025F12028F400374382290026B12028F4033
:2001E3000374392290027712028F4003742A2290028312028F4003742322E4222B434B45C3
:20020300563A2230222C31002B434B45563A2231222C31002B434B45563A2232222C3100B9
:200223002B434B45563A2233222C31002B434B45563A2234222C31002B434B45563A223511
:20024300222C31002B434B45563A2236222C31002B434B45563A2237222C31002B434B4553
:20026300563A2238222C31002B434B45563A2239222C31002B434B45563A222A222C310051
:200283002B434B45563A2223222C310078307B00E66013EB936670090BEB93C3600B084130
:2002A30093087B004193E824CF22758107759870758921758DC2758BC2758780758C8B75B8
:2002C3008A7A752D01D28ED28CD2BB75A81AC20212012B752402D2AF9000261201421201B6
:2002E3002B1200CF90002612014212012B1200DC40301200CA90002B12014212012B12000C
:20030300DC1200CA90003112014212012B1200DC1200CA90004512014212012B1200DC129C
:2003230000CA75240390006712015530B20D200515D2059000611201556149300508C205EE
:20034300900064120155120175B431057524016162B432057524026162B43306752403128B
:05036300012B02032E36
:00000001FF
